:020000040000FA
:020000000528D1
:080008004628812086018501D4
:100010008420FF308500E630860007308100812093
:100020000A30A000053092000C309700861F2C2863
:10003000061F232884200E3092008120083095006E
:100040000130A2003F2884201330920081200A3022
:1000500095000A30A2003F28061F372884201E3052
:10006000920081200F3095001430A2003F28842098
:100070003E30920081201F3095002830A200A10060
:10008000ED3081008B168B1706164528F400030E01
:100090008301F300ED3081000B1D64280B11A008D3
:1000A00003195428A00364280A30A000A108031DE6
:1000B0006328061E5F2806122208A100642806167F
:1000C0002208A1006428A10310140C10730E8300F1
:1000D000F40E740E090084209A0075089B001C150C
:1000E0008B1355309D00AA309D009C148B179C18D3
:1000F00077288120080084209B001C141A08812086
:1001000008008312031308008316031308008312E8
:0A0110000317080083160317080008
:02400E00503F21
:104200000100140064009600FF0020004500320009
:104210002000500075006C0073006500200047000E
:1042200065006E0065007200610074006F0072002E
:10423000200020007700770077002E0063006E00DA
:1042400063002D0065006C0065006B007400720057
:104250006F006E0069006B0061002E006800750041
:1042600020002000260020007700770077002E0035
:1042700068006F0062006200790063006E006300F6
:104280002E00680075002000200026002000770026
:10429000770077002E007100750061006E007400D9
:1042A00075006D0073006500720076006F002E00CF
:0842B00063006F006D002000A7
:00000001FF
